:0200000480007A
:100000006F000005732F2034930F80006308FF03F7
:10001000930F90006304FF03930FB0006300FF038E
:10002000130F000063040F0067000F00732F2034CC
:1000300063540F006F00400093E19153171F0000BD
:1000400023223FFC171F000023200FFC6FF01FFF2F
:100050009300000013010000930100001302000050
:100060009302000013030000930300001304000038
:100070009304000013050000930500001306000020
:100080009306000013070000930700001308000008
:10009000930800001309000093090000130A0000F0
:1000A000930A0000130B0000930B0000130C0000D8
:1000B000930C0000130D0000930D0000130E0000C0
:1000C000930E0000130F0000930F0000732540F102
:1000D0006310050097020000938202017390523072
:1000E000735044749702000093820201739052305F
:1000F00073500018970200009382420273905230AE
:100100009B021000939252039382F2FF7390023B82
:100110009302F0017390023A73504030970200004E
:1001200093824201739052307350203073503030BC
:100130009301000097020000938202ED7390523009
:10014000130510001315F501635C05000F00F00F97
:10015000930110009308D005130500007300000000
:1001600093020000638A020073905210B7B200003D
:100170009B8292107390223073500030372500001C
:1001800073200530735030009702000093824201C3
:1001900073901234732540F17300203093012000D6
:1001A00017250000130505E6071005008710250038
:1001B0000711450083166500532510A4F3151000A0
:1001C00013060000631ED50E639CC50E930130001C
:1001D00017250000130585E307100500871025008B
:1001E0000711450083166500530510A4F315100090
:1001F000130600006316D50C6394C50C93014000F0
:1002000017250000130505E10710050087102500DC
:100210000711450083166500531510A4F31510004F
:1002200013060000631ED508639CC50893015000A7
:1002300017250000130585DE07100500871025002F
:100240000711450083166500532510A4F31510000F
:10025000130600006316D5066394C506930160007B
:1002600017250000130505DC071005008710250081
:100270000711450083166500530510A4F3151000FF
:1002800013060000631ED502639CC5029301700033
:1002900017250000130585D90710050087102500D4
:1002A0000711450083166500531510A4F3151000BF
:1002B000130600006316D5006394C5006310300276
:1002C0000F00F00F638001009391110093E1110082
:1002D0009308D00513850100730000000F00F00F94
:1002E000930110009308D00513050000730000006F
:0C02F000731000C00000000000000000BF
:1010000000000000000000000000000000000000E0
:1010100000000000000000000000000000000000D0
:1010200000000000000000000000000000000000C0
:1010300000000000000000000000000000000000B0
:081040000000000000000000A8
:1020000071BD71BD0000010071BD71BD0000010016
:1020100071BD71BD000000007BBD71BD00000000FE
:102020007BBD71BD000001007BBD71BD00000100E2
:040000058000000077
:00000001FF
